:1000000063C005C805C87AC079C078C077C076C01B
:1000100000C874C073C0AAC571C070C06FC06EC084
:100020006DC00FC66BC029C6BFC6BEC6BDC6BCC6A6
:10003000BBC6BAC6B9C621C6B7C6B6C6B5C6B4C66B
:10004000B3C6B2C6B1C631C6AFC6AEC6ADC6ACC683
:10005000ABC6AAC6A9C63AC6A7C6A6C6A5C6A4C6A2
:10006000A3C6A2C6A1C63BC69FC69EC69DC69CC6C9
:100070009BC69AC699C654C697C696C695C694C6D8
:1000800093C692C691C690C68FC68EC68DC68CC6C4
:100090008BC68AC689C64DC687C686C685C684C62F
:1000A00083C682C681C612C67FC67EC67DC67CC692
:1000B0007BC67AC679C64EC677C676C675C674C67E
:1000C00073C672C671C662C611241FBECFE5D4E0E6
:1000D000DEBFCDBF10E0A0E6B0E0EEEBF0E102C085
:1000E00005900D92A037B107D9F712E0A0E7B0E074
:1000F00001C01D92A43EB107E1F730C091C7089539
:100100008F9A8F9A8A98979887B3807F87BB87B397
:10011000806F87BB84B3807F84BB8EB5887F8EBDA4
:1001200085B78C6085BF85B7836085BF8BB78064DA
:100130008BBF86E083BF85B78F7885BF85B7806822
:1001400085BFE0E0F3E080E3DF01982F1D929A95F0
:10015000E9F7A1E0B0E0182EA0D70895CFE5D4E0EC
:10016000DEBFCDBFCFD6F4D42BD5CADF78947ED6F0
:100170008AD337D288EE93E08AD611D080E090E01F
:100180009DC7F89490917000ECE6F2E0E90FF11D44
:1001900080839F5F9770909370007894089580910A
:1001A0007200882399F080FF07C0F8948E7F8093B7
:1001B00072007894B6D0FFD28091720081FF06C0A1
:1001C000F8948D7F80937200789412D22091710000
:1001D00080917000821719F3F894E22FFF27E459F9
:1001E000FD4F9081822F8F5F87708093710078948C
:1001F000892F9927803131F1813168F48230C9F03B
:10020000833018F4813059F62BC0843031F18830B6
:1002100009F0C5CF1FC0803879F0813820F48032D2
:1002200009F0BDCF14C0813851F0803909F0B7CF43
:100230001CC082E02ED2B3CF80E82BD2B0CF81E8B1
:1002400028D2ADCF80E125D280E175D4A8CF80E25D
:1002500020D2A5CF88E01DD2A2CF84E01AD29FCFB2
:1002600081E069D481E015D29ACF80E964D497CF38
:10027000DF92EF92FF920F931F93CF93DF93209122
:1002800060003091610080917300882309F43FC0C1
:10029000E9018AE05CD28091730059D2DD248F811C
:1002A000813069F588818038E1F0803411F481E093
:1002B00019C0803211F482E015C0803111F483E05E
:1002C00011C0883011F484E00DC0843011F485E051
:1002D00009C0823011F486E005C0813011F487E056
:1002E00001C080E01B810C81FD80EE8030D2812F27
:1002F0002ED2802F2CD28F2D2AD28E2D28D2D3947D
:1003000088E0D81611F02896CACF8FEF20D284E06B
:1003100038DFDF91CF911F910F91FF90EF90DF9029
:1003200008952F923F924F925F926F927F928F9299
:100330009F92AF92BF92CF92DF92EF92FF920F9374
:100340001F93CF93DF93CDB7DEB721970FB6F89405
:10035000DEBF0FBECDBF00916000109161008091A3
:100360007400823009F06AC08BE0FCD38091750084
:10037000F9D30F2EFCEBCF2EF1E0DF2EF02D00E0B5
:1003800010E00F2EFCE0EF2EF1E0FF2EF02DF60135
:100390008081898389818F70898389818295807F1B
:1003A00089839981F70180818F70892B8983898165
:1003B000D9D3D8011196FD01E45FFE4F8081898376
:1003C00089818F70898389818295807F89839981D2
:1003D000A454BE4F8C918F70892B89838981C2D39D
:1003E00082E090E0C80ED91E0E5F1F4FE80EF91E86
:1003F000003B110561F68FE0B5D3809175008F5FEA
:1004000080937500883460F010927500109274002B
:1004100089B78B7F89BF60E081E1E9D4EDD4C8C0A2
:1004200080917200826080937200C2C080E2A9DE77
:1004300089B78B7F89BF10927600BAC0813009F0EE
:10044000B7C0F0907600CF2CDD2436010894610807
:100450007108709173000F2EFCEB2F2EF1E03F2EF0
:10046000F02D50E040E061E0EF2CE394F1013081A9
:10047000560F618182E090E0280E391E460F33232B
:1004800009F45CC0643008F459C0D80120E08C91B4
:100490003817C9F5FD0187818130A9F50F2EF6E0E7
:1004A000AF2EBB24F02DAA0EBB1E86819927861580
:1004B000970549F52D010894411C511C8181882420
:1004C0009924689481F88A0E9B1E9281581710F027
:1004D000951740F4481710F0941720F4851798F0FA
:1004E000491788F0F2015083F4014083FD018381B4
:1004F000581708F45383FD018581841708F4458358
:10050000F501F0821BC02F5F283009F44DC018960A
:10051000BECFD80190E0FD018781882321F0189695
:100520009F5F9830C1F73C93FD0151834283538311
:10053000F4824583F68281E087837F5F403B08F445
:1005400095CF70937300C60187709070079701F57F
:10055000D801179640E08C918130A1F4FD013197CC
:100560009081FD0133978081292F3327F901E81B02
:10057000F10933973CF4C601821B930B039714F0E7
:100580001C9271504F5F1896483029F77093730092
:10059000E0927600F0E9EF1609F448CF80917200FE
:1005A00082608093720004C0783008F4B2CFC6CF66
:1005B00021960FB6F894DEBF0FBECDBFDF91CF916D
:1005C0001F910F91FF90EF90DF90CF90BF90AF9071
:1005D0009F908F907F906F905F904F903F902F9063
:1005E000089580E4E8E7F0E011928A95E9F708952C
:1005F00080917400823049F580917500282F220F78
:1006000080EBECEBF1E0982F11929A95E9F7ECE092
:10061000F1E011928A95E9F7829BFECF829B07C099
:10062000FDCF90E0849BFECF849B04C0FDCF2223AE
:10063000C1F705C09150822F8195981799F76CE00A
:1006400071E08CEB91E0C3D40895813039F4849942
:10065000FECF60E073E08CEB91E072D4089580915E
:1006600074008130A9F41092760080917300809319
:1006700077001092730080E4E8E7F0E011928A9529
:10068000E9F7829BFECF60E073E08CEB91E058D4F9
:100690000895843019F1853028F4813009F18230D1
:1006A00041F507C0803899F0813809F1803209F5A9
:1006B00013C061E081E19BD39FD388EE93E0E7D341
:1006C0001092750082E08093740092DF089581E0BB
:1006D00080937400C4DF0895CBDD0895C0DF0895D2
:1006E00080917400882329F084E04BDD08951092F6
:1006F00074000895DC01862F6623C9F0F8946150D8
:100700006F3FA1F0262F44E952E0861B682F62500C
:100710008091BA00FA01E80FF11D9D9190838F5FDF
:100720008F738093BA002150621791F778940895DF
:10073000F8949091BB00E4E9F2E0E90FF11D8081AB
:100740009F5F9F739093BB00789499270895F894C6
:100750009091BA00E4E9F2E0E90FF11D80839F5F18
:100760009F739093BA00789408959091BA00809105
:10077000BB00981741F0DCDFF5D19091BA00809171
:10078000BB009817C1F708950F931F93CF93DF9382
:10079000EC01862F61506F3F49F0162F861B082F02
:1007A00002508991DFD111500117D9F7DF91CF9114
:1007B0001F910F9108959091BA008091BB009817F6
:1007C00011F0B6DFCFD108959091BF00903541F47C
:1007D0008091C000873409F581E08093620048C0B1
:1007E000973439F48091C000863509F51092620083
:1007F0003FC0943441F48091C000863411F583E009
:100800008093620035C0933441F48091C0008235FA
:1008100011F582E0809362002BC0953441F4809101
:10082000C000843511F584E08093620021C09335C7
:1008300041F48091C0008D34C1F486E08093620061
:1008400017C0943441F48091C000843571F485E080
:10085000809362000DC0923541F48091C0008335D1
:1008600021F487E08093620003C089E080936200F6
:1008700083E0EFEBF0E011928A95E9F71092BE0069
:100880001092BD0008951092BF001092C000109207
:10089000C1001092C20080E4E3ECF0E0982F1192C6
:1008A0009A95E9F7E4E9F2E011928A95E9F780E296
:1008B000E4E7F2E011928A95E9F708958FEB90E072
:1008C000B0D39C018F3F910569F060F089E080937F
:1008D00062008091BC00E3ECF0E0E80FF11D8FEFC7
:1008E000808307C08091BC00E3ECF0E0E80FF11DCD
:1008F000208383E0EFEBF0E011928A95E9F7109204
:10090000BE001092BD000895FF920F931F93CF93E6
:10091000DF930F2EF9E0FF2EF02DFFC0F894E22FA9
:10092000FF27EC58FD4F9081822F8F5F8F7180934E
:10093000B90078949D3009F0B1C08091BC00882343
:1009400011F442DF06C0BADF8091BC008F5F809354
:10095000BC0084E690E09BD2809162008850823097
:1009600058F48EE4F4DE83E4F2DE8BE4F0DE8DE016
:10097000EEDE80E906DC89C081E4E9DE83E4E7DEBF
:100980008BE4E5DE8DE0E3DE80E9FBDB8091620055
:10099000813009F47AC0882371F480916300882340
:1009A00009F473C0C3E6D0E02196D1DE88818823A4
:1009B00009F46BC0F9CF873011F4A1DB66C0833036
:1009C00031F484E690E063D282E0DBDB5EC082300B
:1009D00099F48091BC00823068F011E0E12FFF278C
:1009E000ED53FF4F6181808102D21E5F8091BC0078
:1009F0001817A0F301D249C0843031F484E690E0A6
:100A000046D280E8BEDB41C0853019F481E8B9DB0D
:100A10003CC0863009F039C08091BC00882309F4BD
:100A200034C040E003EC10E060E073E0842F9927CD
:100A30009C012F5F3F4FF901E00FF11FE081EC01B6
:100A4000C60FD71FE883D90120D3802DE817C1F046
:100A5000D9010E2E27D3D90118D3802D988198174C
:100A600079F0D901092E1ED3D9010FD3802D988199
:100A7000981731F0D901092E15D3D90106D3802D4D
:100A80004F5F8091BC00481788F21092BC0080E450
:100A9000E3ECF0E011928A95E9F73FC09032F1F46F
:100AA0008091BC00882339F48FDE8091BC008F5F79
:100AB0008093BC0032C09927CF974CF01092BD00B4
:100AC0001092BE001092BC00F092620026C0F6DECA
:100AD0008091BC008F5F8093BC001FC0892F815420
:100AE0008A3118F08F5E8A30B0F48091BE00E82F12
:100AF000FF27E154FF4F90839091BD009F5F90933B
:100B0000BD008F5F8093BE00943038F0F092620099
:100B10001092BE0002C0F09262002091B900809154
:100B2000B800821709F0FACEE894DF91CF911F91B7
:100B30000F91FF900895803129F0803939F081308C
:100B400031F402C038DE0895DFDE08950EDE089528
:100B500010BC82E189B988E98AB986E880BD82E063
:100B60008BB908955D9BFECF8CB908951F920F92AB
:100B70000FB60F9211248F939F93EF93FF93809161
:100B8000B8009CB1E4E7F2E0E80FF11D90838F5FBD
:100B90008F718093B80080917000ECE6F2E0E80F6E
:100BA000F11D91E090838F5F877080937000FF91BB
:100BB000EF919F918F910F900FBE0F901F901895FE
:100BC00011B888E480B90895982F8091080188238E
:100BD000E4F306B604FCFDCF909303017093050186
:100BE00060930401409307011092060110920901DD
:100BF00085EA86BF80910801806880930801089586
:100C0000982F809108018823E4F390930301709357
:100C10000501609304014093070181E08093060180
:100C20001092090185EA86BF80910801806880934F
:100C30000801089580910801881F8827881F992737
:100C400008951F920F920FB60F9211248F939F93C6
:100C5000AF93BF93EF93FF9381B19927AA27BB2747
:100C6000887F9070A070B070FC013897E135F10575
:100C700008F09AC0ED5EFF4F09948091090183301E
:100C800048F086B7806986BF809108018F7780938E
:100C900008018AC08091030190910601880F890F95
:100CA00083B986B78F7D86BF7FC010920901E0911E
:100CB0000401F0910501808183B93196F09305011B
:100CC000E093040186B7806886BF6EC080910901F9
:100CD0008F5F8093090186B7806B86BF65C0809166
:100CE000070181508093070180910701882379F0E3
:100CF000E0910401F0910501808183B93196F09370
:100D00000501E093040186B7806886BF4DC086B7B1
:100D1000806986BF809108018F778093080144C065
:100D200086B7806986BF809108018F77809308011C
:100D30003BC080910701815080930701809107019A
:100D4000882321F086B7806C86BF2EC086B7806866
:100D500086BF2AC0E0910401F091050183B1808330
:100D60003196F0930501E0930401809107018150D1
:100D70008093070180910701882321F086B7806C5A
:100D800086BF12C086B78F7B86BF0EC0E09104017C
:100D9000F091050183B1808386B7806986BF809119
:100DA00008018F7780930801FF91EF91BF91AF9178
:100DB0009F918F910F900FBE0F901F9018952091CB
:100DC0000A01E22FFF27EE0FFF1FEC52FD4F918328
:100DD00080832F5F277020930A0190E080910B01A0
:100DE000281709F491E081E0892799270895282F91
:100DF000362FC901E4DF08950F931F93CF93DF933C
:100E0000CDB7DEB722970FB6F894DEBF0FBECDBFC9
:100E10008E010F5F1F4F19C0E32FFF27EE0FFF1F3B
:100E2000EC52FD4F91812081832F8F5F87708093DB
:100E30000B019A83298342E0B80180E6C5DE84E68F
:100E400090E025D0F7DE8130E9F330910B018091FD
:100E50000A01831709F722960FB6F894DEBF0FBE7A
:100E6000CDBFDF91CF911F910F91089560E284E192
:100E7000BEDF60E489E3BBDF68E282E1B8DF65E002
:100E800088E2B5DF61E083E1B2DFB6DF0895CF939A
:100E9000DF93CDB7DEB724970FB6F894DEBF0FBE51
:100EA000CDBF9C011A8219821C821B821A82198270
:100EB00089819A8182179307E0F41C821B828B81BF
:100EC0009C81885E934058F400008B819C81019640
:100ED0009C838B838B819C81885E9340A8F389815E
:100EE0009A8101969A83898389819A8182179307CF
:100EF00020F324960FB6F894DEBF0FBECDBFDF916E
:100F0000CF9108958E9A969A84EF91E0C0DF9698DB
:100F100084EF91E0BCDF969A84EF91E0B8DF969879
:100F200084EF91E0B4DF969A84EF91E0B0DF969879
:100F300084EF91E0ACDF969A0895969A96988895FA
:100F4000E6F13EB537603EBD00E010E520E0B92F88
:100F5000A82FF72FE62FD72F39B7346039BF30E5E8
:100F60004FEF4DBD3CBDC62F3BB730683BBF969A97
:100F7000889596983BB73F773BBF00000000E6B3EB
:100F8000C3B3CF703081E6B3488950A134233523F1
:100F900076F03217A1F3969A00009698412F0CB57F
:100FA000102F041B2D930D93232F0000E8CF0FEF7C
:100FB000011B03953D930C9300C03EB5387F3EBDA9
:100FC000969A9698E8940895969A96988895AEF38E
:100FD000B92FA82FD72FC62F30E54FEF4DBD3CBD01
:100FE0003EB537603EBD000039B7346039BF3BB70E
:100FF00030683BBF969A889596983BB73F773BBF42
:10100000000033B346B33D934993DEF7D6CF18952E
:101010001895309172003160309372006894189581
:101020001895FC0188279927E89421912223E9F05B
:101030002032D9F32930C9F32A30B9F32C30A9F37F
:101040002D3099F3263789F32B3219F02D3221F404
:1010500068942191222349F020333CF02A332CF468
:1010600020530BD0820F911DF4CF8115910521F0F3
:101070001EF480959095019608957AE0979F902DA3
:10108000879F802D910D11240895E199FECFBFBB5C
:10109000AEBBE09A11960DB20895F7DF01921A9453
:1010A000E1F70895E199FECFBFBBAEBB0DBA119633
:0E10B0000FB6F894E29AE19A0FBE0895FFCFB2
:1010BE0078000841565263616D2076312E340D0052
:00000001FF
